:1000000085C200009FC200009DC200009BC200008C
:1000100099C2000097C2000095C2000093C2000080
:1000200091C200008FC200008DC200008BC2000090
:1000300089C2000087C2000085C2000083C20000A0
:1000400081C200007FC200007DC200007BC20000B0
:1000500079C20000D9C3000075C2000073C200005D
:1000600071C200006FC200006DC200006BC20000D0
:1000700069C2000067C2000065C2000063C20000E0
:1000800061C200005FC200005DC200005BC20000F0
:1000900059C2000057C2000055C2000053C2000000
:1000A00051C200004FC200004DC200004BC2000010
:1000B00049C2000047C2000045C2000043C2000020
:1000C00041C200003FC200003DC200003BC2000030
:1000D00039C2000037C2000035C2000033C2000040
:1000E00031C20000A0A1A1A01B09A51CA010A0A0C6
:1000F000201A0111B12C0D0E02160318A00B0A08CC
:1001000007060413A009151914120517A0A6A40DBB
:100110000A0F0CA0A01D1BA0A0C0BFBE00BDBCBB91
:10012000BAB9B8B7A8A9AAAB0000ADACA0A1A1A06C
:100130001B09A55C7F503B2F205A4151A02C4D4EEE
:1001400042564358A04B4A4847464453A049555944
:1001500054524557A0A6A40D0A4F4C2E7E5D5B2D30
:100160003A3039384037363534333231A8A9AAAB62
:100170000000ADACA0A1A1A01B09A57C7F502B3F26
:10018000205A4151B23C4D4E42564358A04B4A482A
:1001900047464453A049555954524557A0A6A40D6B
:1001A0000A4F4C3E7E7D7B3D2A302928602726253C
:1001B00024232221A8A9AAAB0000ADACA0A1A1A034
:1001C0001B09A55C7F703B2F207A6171A02C6D6E9E
:1001D00062766378A06B6A6867666473A0697579F4
:1001E00074726577A0A6A40D0A6F6C2E7E5D5B2DE0
:1001F0003A3039384037363534333231A8A9AAABD2
:100200000000ADACA4A1A1A0A01BA515A010A0A0AA
:10021000201A0111A02C0D0E02160318A00B0A08BB
:1002200007060413A009151914120517A0A0A00DA4
:10023000A60F0CA0A0A0B1A0A0C0BFBE08BDBCBBB3
:10024000BAB9B8B7A8A9AAAB0000ADACA4A1A1A047
:10025000A01BA515A0503B2F205A4151A02C4D4E5C
:1002600042564358A04B4A4847464453A049555923
:1002700054524557A0A0A00DA64F4C2EA0A0A02DD3
:100280003A3039380837363534333231A8A9AAAB79
:100290000000ADACA4A1A1A0A01BA515A0402B3FC0
:1002A000205A4151A03C4D5E42564358A04B4A480B
:1002B00047464453A049555954524557A0A0A00D54
:1002C000A64F4C3EA0A0B23D2A302928082726255B
:1002D00024232221A8A9AAAB0000ADACA4A1A1A00F
:1002E000A01BA515A0502B3F205A4151A03C4D4EBC
:1002F00042564358A04B4A4847464453A049555993
:1003000054524557A0A0A00D404F4C3EA0A0B23D76
:100310002A3029280827262524232221A8A9AAAB88
:100320000000ADACA4A1A1A0A01BA5157F703B2F20
:10033000207A6171A02C6D6E62766378A06B6A681A
:1003400067666473A069757974726577A0A0A00D63
:100350005E6F6C2EA0A0A02D3A30393808373635A4
:1003600034333231A8A9AAAB0000ADACA5A2011369
:10037000040607080A0B0C0B0A7FB1A5A4A11A18E2
:100380000316020E0D0C0E0FA180A0A01B0102038C
:10039000040506070809000D1E1B1C1DB2091117D4
:1003A0000512141915090F10000D0A8CA8A9AAAB83
:1003B0000000ADACB3978120939A8E8B2D372A38ED
:1003C0002F39A0A0343135323633A0A0302E2BA0E7
:1003D000A0A0A0A0A5A24153444647484A4B4C3B8D
:1003E0003A5FA6A5A4A15A584356424E4D3C3E3F03
:1003F000A180A0A01B212223242526272829203DD7
:100400007E5B5C5DB20951574552545955494F5076
:10041000600D0A8CA8A9AAAB0000ADACB3978120EF
:10042000939A8E8B2D372A382F39A0A0343135324C
:100430003633A0A0302E2BA0A0A0A0A0A5A241538F
:10044000444647484A4B4C3B3A7FA6A5A4A15A587C
:100450004356424E4D2C2E2FA180A0A01B3132338B
:10046000343536373839302D5E5B5C5DB209515713
:100470004552545955494F50400D0A8CA8A9AAAB72
:100480000000ADACB3978120939A8E8B2D372A381C
:100490002F39A0A0343135323633A0A0302E2BA016
:1004A000A0A0A0A0A5A26173646667686A6B6C3B9C
:1004B0003A7FA6A5A4A17A786376626E6D2C2E2F62
:1004C000A180A0A01B313233343536373839302D76
:1004D0005E5B5C5DB20971776572747975696F7086
:1004E000400D0A8CA8A9AAAB0000ADACB39781203F
:1004F000939A8E8B2D372A382F39A0A0343135327C
:100500003633A0A0302E2BA0A0A0A0A011241FBE87
:10051000CFEFD1E2DEBFCDBF13E0A0E0B2E0E8EE66
:10052000F9E102C005900D92A033B107D9F724E09C
:10053000A0E3B3E001C01D92A43CB207E1F71AD7D3
:100540000C94C40C5DCD805A813208F037C0E82F7E
:10055000F0E0EA53F34F31C7CEC3CFC3D2C3D6C303
:10056000E1C3E9C47EC385C38CC393C3B0C1CBC40C
:1005700087E06CC588E06AC589E068C581E066C52A
:1005800082E064C583E062C584E060C585E05EC545
:1005900086E05CC584E0D2C285E0D0C286E0CEC2EF
:1005A00087E0CCC288E0CAC289E0C8C28AE0C6C27D
:1005B0008BE0C4C28CE0C2C28DE0C0C20895815AF3
:1005C0008D3070F4E82FF0E0E951F34FF6C6AEC37A
:1005D000AFC3C9C442C349C350C357C37BC17FC45F
:1005E0000895682F8091330345C2CF93C82F813A75
:1005F00018F0A9DFCF910895F4DF809134038C17B0
:10060000C9F3C093340362D4F5CFCF93C82F8A3097
:1006100041F06C2F809132032DD28C2F90E0CF913E
:1006200008958DE0F2DFF5CFCF938091320355D25C
:10063000C82F803A41F080913003909131035CD112
:100640008C2FCF9108958091330347D2C82FF8CFD4
:1006500090E090933103809330030895CF93DF931C
:10066000C82FD62F68D3482F6D2F8C2F16D3DF912C
:10067000CF9108956F927F928F929F92AF92BF9287
:10068000CF92DF92EF92FF920F931F93CF93DF935E
:1006900081E063D2A82EB92E83E050D200E00F2E65
:1006A000FAE07F2EF02D88248394912C0F2EF0EA0F
:1006B0006F2EF02D5AC08C2F90E0F701E80FF91F34
:1006C00020813FEF320F2130D1F03083D69516953F
:1006D000CF5F94D2C81708F047C0D0FDECCF10FF11
:1006E000F5CF6C2F802FBADF909134038913EECFB2
:1006F00047D4882359F38091340377DFE7CFF7019C
:10070000E80FF91F708210FF12C0F601EB54FC4F86
:1007100094010C2E02C0220F331F0A94E2F780814D
:10072000822B80836C2F802F99DF5FDFCFCFF60184
:10073000EB54FC4F94010C2E02C0220F331F0A947D
:10074000E2F7C90180959081892380836C2F802FE7
:1007500085DF813A38F4909134038913B7CF6092E2
:100760003403B4CF2CDFB2CF0F5F3DD20817C0F4F3
:10077000802FF5010995182FC02ED12CF601EB54CE
:10078000FC4FD081D827C0E0C601880F991F880F81
:10079000991F880F991F9C012B5C3C4F790199CFC1
:1007A000DF91CF911F910F91FF90EF90DF90CF904D
:1007B000BF90AF909F908F907F906F90089580EA48
:1007C0008093340314D173D346D280E190E022D1D8
:1007D0008093330380E890E01DD180933203A5EB32
:1007E000B3E0E5E3F3E025EC33E08AE01D9280839B
:1007F00081838283838384838583868387833896FA
:100800002A173B0799F708958F9381E08093C603D9
:100810008F9118958091C6031092C603089588237E
:1008200011F05D9808955D9A0895882311F05E98FF
:1008300008955E9A0895882311F05F9808955F9A4D
:1008400008950895882319F02D9A259A08952D98D2
:10085000FCCF882319F025982D9A08952D98259A74
:100860000895882319F02D9A259A089525982D9892
:100870000895882319F02E9A269A08952E98FCCF71
:10088000882319F026982E9A08952E98269A08956E
:10089000882319F02E9A269A089526982E9808955E
:1008A000882319F02F9A279A08952F98FCCF882330
:1008B00019F027982F9A08952F98279A089588233A
:1008C00019F02F9A279A089527982F9808952C9811
:1008D000249A08952C9A249A089585E38A95F1F72D
:1008E000000008952FEF80E792E021508040904073
:1008F000E1F700C000000895282F392F2115310598
:1009000061F080E090E0EFE9FFE03197F1F700C09F
:100910000000019628173907B1F70895CF93F8948E
:100920001092C60387E0809361001092C60389EF9E
:1009300087BD15BC82E084BD80936E0083E085BDD9
:100940008091C50380930201CFEFC0930101109203
:10095000C503BDDF559A569A579AC1B9C093040191
:1009600017B8C8B97894CF910895282F81E090E006
:10097000A0E0B0E004C0880F991FAA1FBB1F2A95F2
:10098000D2F780959095A095B0958093050125E1CB
:100990002A95F1F70000892F9A2FAB2FBB2782B938
:1009A00085E18A95F1F7000086B1809508959091D0
:1009B000C5038927809302011C9A85E38A95F1F784
:1009C00000001C9A0895833059F028F4813039F0E2
:1009D000823021F4FAC3843009F48EC487C3B8C3CB
:1009E00027C4982F81E0953008F080E00895109298
:1009F000C9031092C8031092C7030895882344F0D6
:100A000091E02091C70382170CF090E0892F0895A0
:100A100080E00895282F392F8091C703843034F562
:100A20006091C8037091C90340E950E0461B570B21
:100A300042175307ECF091E0980F9093C70397E0AB
:100A40008902F0011124E653FC4F33832283AB016A
:100A50004A515C4F51834083148215821682260FBF
:100A6000371F3093C9032093C80308958FEF08956B
:100A70008FEF0895CF93DF93C82FD62FBFDF882342
:100A800049F18C2F0C2E000C990B27E0C202F001CB
:100A90001124E653FC4F268162817381422F50E07E
:100AA00046175707BCF4FC01EE0FFF1FEE0FFF1FA8
:100AB000EE0FFF1FE81BF90BE653FC4F848190E01B
:100AC000A081B181A80FB91FDC93019663D4848300
:100AD0002F5F2683DF91CF910895CF93C82F8EDFAC
:100AE00030EA882339F18C2F0C2E000C990B27E06B
:100AF000C202F0011124E653FC4F268130EA222382
:100B0000C9F0FC01EE0FFF1FEE0FFF1FEE0FFF1FDE
:100B1000E81BF90BE653FC4F858190E0A081B18181
:100B2000A80FB91F3C9101966281738133D48583EC
:100B300021502683832FCF91089508959FEF980F1A
:100B40009D3050F4E82FF0E0EE0FFF1FEA58FB4F06
:100B50000190F081E02D099508959FEF980F9D3049
:100B600048F4E82FF0E0EE0FFF1FEA58FB4F8081BA
:100B7000918108958DE995E008959FEF980F9D303C
:100B800040F4E82FF0E0EE0FFF1FEA58FB4F6083C0
:100B900071830895E6E7F4E022E934E08DE995E019
:100BA00081939193E217F307D9F7E6E7F4E085EB39
:100BB00094E09383828387ED94E095838483089502
:100BC000643080F4413170F4293060F4E62FF0E0B5
:100BD000EE0FFF1FEE0FFF1FED56FB4F808391833B
:100BE000428323830895A7D0E82FF0E0EE0FFF1F84
:100BF000EE0FFF1FED56FB4F828108959CD0E82F2A
:100C0000F0E0EE0FFF1FEE0FFF1FED56FB4F83814D
:100C10000895CF93DF93D82FE4DE811103C0DF91D5
:100C2000CF910895D093920479DEC0E020E040E0B7
:100C30006C2F80E090E0C4DFCF5FC430B9F731D2D1
:100C4000A9DF8D2FC0DEEBCF90919204981301C0E5
:100C50000895DFDFFDCF80E0DCCF809192048E7FAE
:100C6000F3CF809192048160EFCF809192048D7FC9
:100C7000EBCF809192048260E7CF809192048B7FCA
:100C8000E3CF809192048460DFCF80919204877FCC
:100C9000DBCF809192048860D7CF982F2091920467
:100CA00030E0F901EE0FFF1FEE0FFF1FED56FB4F77
:100CB00083818823C1F022812223A1F0E42FF0E078
:100CC000EE0FFF1FEE0FFF1FED56FB4F70E0899FE9
:100CD000600D711D11240190F081E02DE60FF71FCA
:100CE00084910895822F08958093A50461E081FF87
:100CF00062E08BE074C181E0F7CF8091A50482604F
:100D0000F3CF8091A50492E08927EECF9091A404BF
:100D100081E089278093A40461E0913009F462E0C6
:100D20008AE05DC181E08093A304089580E0DCCF78
:100D30001092A3040895E1E08091A504811101C0FF
:100D4000E0E08091A4048111E2608091A30481110C
:100D5000E460F0E0EE5BFD4F808108951F93CF9338
:100D6000DF93162FC82FD0E0CC0FDD1FCC0FDD1F77
:100D7000C050DE4FE881F981862F09951A83DF91F3
:100D8000CF911F910895CF93DF93C82FD0E0CC0F60
:100D9000DD1FCC0FDD1FC050DE4FE881F98181E0FF
:100DA000099581E08A83DF91CF910895CF93DF93F6
:100DB000C82FD0E0CC0FDD1FCC0FDD1FC050DE4FA1
:100DC000E881F98180E009951A82DF91CF91089539
:100DD000E82FF0E0EE0FFF1FEE0FFF1FE050FE4F79
:100DE00061E09281911160E0B9CF282F90910302C8
:100DF0009923B9F0981779F0E92FF0E0892FEE0FD9
:100E0000FF1FEE0FFF1FE050FE4F9381992359F013
:100E10002913F2CF0895882311F080E008958DE022
:100E200008958DE008958DE00895E82FF0E0EE0F2D
:100E3000FF1FEE0FFF1FE050FE4F838108951F93A9
:100E4000CF93DF93C82FD62F142FCFDF9FEF9C0FA8
:100E50009C30C8F48D30E1F0EC2FF0E0EE0FFF1F76
:100E6000EE0FFF1FE050FE4F9381A82FB0E0AA0FB6
:100E7000BB1FAA0FBB1FA050BE4F13969C93D383DA
:100E8000128381E001C080E0DF91CF911F9108952E
:100E900080E0FACFE2E0F2E080E091E090838F5FC3
:100EA000818334968D30D1F71092330208958DE00E
:100EB00092E09093A9048093A8049093AB0480934C
:100EC000AA049093A7048093A60408958091AA048D
:100ED0009091AB049093A7048093A6040895109278
:100EE000A9041092A8048091AA049091AB048234C2
:100EF000910541F01092AB041092AA041092A7043D
:100F00001092A60408958DE092E09093A904809336
:100F1000A8048091AA049091AB048234910551F009
:100F20008DE092E09093AB048093AA049093A70481
:100F30008093A60408958091A6049091A704833419
:100F4000910530F48091AA049091AB04892B51F45F
:100F500082E490E09093AB048093AA049093A7045A
:100F60008093A60408958091A8049091A904909379
:100F7000AB048093AA049093A7048093A6040895D9
:100F80008091A6049091A704009799F09C012150AC
:100F90003109019731F03093A7042093A60480E033
:100FA000089582E490E09093A7048093A60481E0E2
:100FB000089580E008950F931F93CF93082F192F62
:100FC000C62F662341F08C2FF80109958C2F2DDF59
:100FD000C82F8111F8CFCF911F910F910895CF9312
:100FE000E82FF0E0EE0FFF1FE455FB4FC0816330A8
:100FF000F1F048F0643081F06530B9F46C2F88EE80
:1010000096E0D9DF12C06130E1F0623071F46C2FEC
:1010100086ED96E0D0DF09C06C2F88EE96E0CBDF3E
:1010200061DC6C2F88EE96E0C6DFCF9108956C2FBF
:1010300088EE96E0C0DF51DC6C2F88EE96E0BBDFD7
:10104000F4CF6C2F83EC96E0B6DFEFCFE82FF0E023
:10105000EE0FFF1FE455FB4F6181C1CF0F931F932C
:10106000CF93DF93162F042F9FEF980F9B3028F01C
:10107000DF91CF911F910F910895C82FD0E0FE010D
:10108000EE0FFF1FE455FB4F422F6081812FD7DE0B
:10109000882371F3CC0FDD1FC455DB4F1883098300
:1010A000E7CFF8DEECEAF4E084EC94E01182108201
:1010B0003296E817F907D1F70895CF93DF93CDB7AC
:1010C000DEB7AE014B5F5F4FFA0161917191AF01E5
:1010D00084E392E08CD1DF91CF9108958AE492E08D
:1010E0009F938F93EADF0F900F90089588E2B0DA14
:1010F00060E080E057D062E081E054D061E082E0BF
:1011000051D063E083E04ED06EE678E08DE035DDCF
:1011100062E479E08CE031DD21E040E06AE087E0E4
:101120009DDF20E040E06CE08AE098DF21E043E0D2
:1011300068E081E093DF20E044E063E082E08ECF6E
:101140008AE492E09F938F93B8DF0F900F900895F9
:1011500088E27EDA60E081E025D062E081E022D0A2
:1011600061E082E01FD063E083E01CD060EA78E0B9
:101170008DE003DD62E479E08CE0FFDC21E040E01B
:101180006AE087E06BDF20E040E06CE087E066DF4C
:1011900021E043E068E081E061DF20E044E063E0DB
:1011A00082E05CCFE82FF0E0EE0FFF1FE35AFD4F27
:1011B00028E049E08081918103CD85E692E09F930C
:1011C0008F937BDF0F900F90089588E241DA60E003
:1011D00080E07FD062E081E07CD061E082E079D085
:1011E00063E084E076D062E479E08CE0C6DC6DED0B
:1011F00078E08DE0C2DC20E040E06AE08AE02EDFAB
:1012000020E040E06CE088E029DF21E043E068E096
:1012100081E024DF20E044E063E082E01FDF76CD60
:1012200082E892E09F938F9348DF0F900F9008958C
:1012300088E20EDA60E081E04CD062E081E049D0E3
:1012400061E083E046D063E084E043D062E479E08B
:101250008CE093DC60E179E08DE08FDC20E040E021
:101260006AE087E0FBDE20E040E06CE088E0F6DE4C
:1012700021E043E068E081E0F1DE20E044E063E06B
:1012800082E0ECCE89E992E09F938F9316DF84EAA7
:1012900092E09F938F9311DF84EB92E09F938F9363
:1012A0000CDF8EED92E09F938F9307DF84EF92E047
:1012B0009F938F9302DF8AE093E09F938F93FDDEED
:1012C0008DB79EB70C960FB6F8949EBF0FBE8DBF1C
:1012D0000895E82FF0E0EE0FFF1FEA5EFC4F28E0D4
:1012E00049E0808191816CCC80E293E09F938F9361
:1012F000E4DE0F900F90089528E04DE060E084EA6E
:1013000094E05EDC28E04DE062E08CE394E058DCA1
:1013100028E04DE061E084ED93E052DC28E04DE010
:1013200063E08CE693E04CDC88E292D920E040E078
:101330006AE08AE093DE20E040E06CE08BE08EDE45
:1013400021E045E061E083E089DE20E045E06BE0FC
:1013500083E084DE21E043E068E081E07FDE21E09D
:1013600044E064E082E07ADED1DCB4DA64E779E07C
:101370008DE003CC24DA01C07DD94CDA8823E9F36F
:1013800053D9C82F803AC1F382E0E7DBFC018C2FF0
:101390000995F2CF97FB072E16F4009406D077FD3F
:1013A00008D011D007FC05D03EF4909581959F4F51
:1013B0000895709561957F4F0895EE0FFF1F05907A
:1013C000F491E02D0994AA1BBB1B51E107C0AA1F91
:1013D000BB1FA617B70710F0A61BB70B881F991FD6
:1013E0005A95A9F780959095BC01CD010895AFE07D
:1013F000B0E0ECEFF9E094C26C017B018A01DC0102
:1014000017961C921E92169713968C9181FFDEC13F
:101410002AE0522EF6019381F70193FD859193FF07
:1014200081917F01882309F471C0853239F493FDDD
:10143000859193FF81917F01853221F4B60190E07F
:10144000DED1E8CF912C612C712CFFE1F71508F467
:1014500045C08B32C1F1F0F48032B9F1833209F426
:101460003AC0833609F487C0833709F490C08335C6
:1014700009F0B0C0F801A190B1908F01692D70E022
:1014800076FC02C06FEF7FEFC501A3D14C016894D9
:1014900077F85EC08D32E1F0803351F020ED280FF7
:1014A0002A3048F18E3209F038C0689476F802C0CC
:1014B000689470F8F70193FD859193FF81917F0106
:1014C0008111C3CF32C0689471F8689472F8F2CF7A
:1014D000689473F8EFCF689474F8ECCF77FC25C06C
:1014E00020ED280F2A3070F476FE05C0959C200D63
:1014F0001124922EDFCF659C200D1124622E68945A
:1015000075F8D8CF8E3249F476FECFCFD601169635
:101510008D919C912F96EFE01FC28C3619F4689440
:1015200077F8C8CF883609F4C5CF982F9F7D95549A
:10153000933008F096CF0C5F1F4F8FE38983882488
:101540008394912CAE014F5F5F4F5A01E89477F876
:1015500073FC05C0862D90E08816990630F1811441
:10156000910449F5662009F455CFB60180E290E078
:1015700046D16A94F7CFD8018C9189830E5F1F4FB3
:1015800088248394912CFE0131965F01DFCFD8012E
:10159000AD90BD908D01692D70E076FC02C06FEFBB
:1015A0007FEFC50121D14C01D1CFB60180E290E09F
:1015B00026D16A94CFCFF50177FC859177FE819192
:1015C0005F01B60190E01BD161106A94F1E08F1ABF
:1015D0009108C5CF843619F0893609F07DC0F8012D
:1015E00077FE73C061917191819191918F01272D47
:1015F0002F76822E97FF09C0909580957095619502
:101600007F4F8F4F9F4F689487F82AE030E0AE01FC
:101610004F5F5F4F5A0123D18A19A82EBA2C782C1C
:1016200086FE0CC0E89470F8A91440F484FE05C04E
:1016300082FC03C0782D7E7E772EB92C74FEA1C06B
:10164000FE01EA0DF11D8081803309F093C0872DE2
:10165000897E782E73FC0EC070FEA1C09A2CB61441
:1016600018F4960C9B18B62C862D8B196B1408F465
:1016700080E0B80EB61408F094C06B1874FE93C0E6
:10168000B60180E390E0BBD072FE08C088E590E030
:1016900071FC02C088E790E0B601B1D0A91408F44B
:1016A0008FC0AA94B12C9FEFA91AB90ADE01119636
:1016B0004D01AA0EBB1EF50182915F01B60190E0BB
:1016C0009ED08A149B04B9F74DCF61917191072E7A
:1016D000000C880B990B8ACF872CE89484F82AE0B9
:1016E00030E0853769F0572D597F852E803769F1B5
:1016F00010F5883569F18F3609F008CF28E030E021
:10170000F80187FE2DC081919191A191B1918C87B3
:101710009D87AE87BF878F01BE016F5F7F4F5B01E3
:10172000AB016C857D858E859F8599D08A19A82E01
:10173000E89487F873CF883709F0E8CE84FE02C0BA
:10174000689482F820E130E0DBCF689484F8F6CF2B
:1017500074FE03C0652F6660862E20E132E0D0CF94
:1017600081919191AC0160E070E04C875D876E875C
:101770007F87D1CF72FC02C0B3946CCFB394B39483
:1017800069CF872D8678882309F464CFF5CFB60119
:1017900080E290E034D083948614C8F365CF8B2C1C
:1017A000FBCF612C6BCF872D8678882309F476CF09
:1017B0008BE271FE80E277FC8DE2B60190E06DCFA6
:1017C000B60180E390E01BD09A9468CF8FEF9FEF33
:1017D000A1CEFC010590615070400110D8F78095B2
:1017E00090958E0F9F1F0895FC01615070400190ED
:1017F0000110D8F7809590958E0F9F1F08950F9335
:101800001F93CF93DF93182F092FEB018B8181FD5D
:1018100009C01FEF0FEF812F902FDF91CF911F9104
:101820000F91089582FF14C02E813F818C819D818C
:10183000281739073CF4E881F981CF010196998393
:10184000888310838E819F8101969F838E83E3CF4F
:10185000E885F985812F0995892BA1F3DACFFA0163
:10186000AA27283051F1203181F1E8946F936E7FDF
:101870006E5F7F4F8F4F9F4FAF4FB1E03ED0B4E0D0
:101880003CD0670F781F891F9A1FA11D680F791F11
:101890008A1F911DA11D6A0F711D811D911DA11D22
:1018A00020D009F468943F912AE0269F1124301932
:1018B000305D3193DEF6CF010895462F4770405DCD
:1018C0004193B3E00FD0C9F7F6CF462F4F70405D7C
:1018D0004A3318F0495D31FD4052419302D0A9F7D7
:1018E000EACFB4E0A6959795879577956795BA95D1
:1018F000C9F700976105710508959B01AC010A2E97
:1019000006945795479537952795BA95C9F7620F6D
:10191000731F841F951FA01D08952F923F924F9211
:101920005F926F927F928F929F92AF92BF92CF926F
:10193000DF92EF92FF920F931F93CF93DF93CDB778
:10194000DEB7CA1BDB0B0FB6F894DEBF0FBECDBFF0
:1019500009942A88398848885F846E847D848C84C1
:101960009B84AA84B984C884DF80EE80FD800C81CA
:101970001B81AA81B981CE0FD11D0FB6F894DEBFAD
:101980000FBECDBFED010895F894FFCFCA02AC029F
:10199000AD02AE02AF02B002B102CA02B202B3029D
:1019A000B402B502B702B602B802BA02BC02BE0265
:1019B000C002C202C402C602C802CA02CC02CE02DF
:1019C000D002D202D402D602D802DA02DC02E70246
:1019D000F002F002F002E802E902F002EA02EB0291
:0819E000EC02ED02EF02EE0241
:1019E8002104000022040000290400003104000042
:1019F80039040000400400004804000050040000BE
:101A0800570400005F0400000F04000015040000E4
:101A18001B04000000000002000000000503000095
:101A2800000000010201030303035B4B65796D614C
:101A3800703A20636C61737369635D0A00BC012CA2
:101A4800017401E4005B4B65796D61703A20417067
:101A5800706C6520322028752F6C206361736529AE
:101A68005D005B4B65796D61703A204170706C6503
:101A7800203220434150535D0031302047455420E7
:101A880041240D0032302041203D2041534328415C
:101A980024290D0033302049462041203C20333290
:101AA800205448454E2041243D2243544C2B222BA0
:101AB800434852242841202B203634290D00343045
:101AC800203F2227223B41243B2227203D20223B46
:101AD800413A0D0035302049462041203C3E203314
:101AE80020474F544F2031300D00363020454E44AA
:101AF8000D52554E0D0024034C02DC0294020402E0
:101B08005B4B657962643A20536F6C2D32305D000F
:00000001FF
